:020000040000FA
:0400000000005E2876
:08000800F300030E8301F10077
:100010000A08F2008A11F124B51C29281F151F199E
:100020000F28840A831603131E088007840303180D
:10003000800A831203131E088007840A840AC90BEE
:100040002F28A03084001430C900EA0B2F28B510E7
:100050003510351C2F28013036020319B5148316CC
:10006000CB0F55288301050883163439C90048028F
:10007000031C4B28031D532834304902031953280D
:10008000CC0B532883125030351D08308316CC001A
:100090008312351653284808CA0083125030351D84
:1000A00008308316CC004908C80083010C1172087F
:1000B0008A00710E8300F30E730E0900831203137E
:1000C0008B018A01850186018701F401B501903019
:1000D00087003515B5157414AA012A170130EF00F1
:1000E000F0008316031385309F00FF3085008312D4
:1000F000031381309F0083160313C0308600013044
:1001000087003430C800CA00CB015030CC00CD018C
:10011000112511251125831203130330C300860016
:10012000861600000000000086121125C30B9028DF
:10013000023086005725283034250C30342506300F
:100140003425762561250519CF28B428051E1526E6
:10015000851E1A260519A628351DAF283626D10A70
:100160005108023C031DB528D101351161254130EC
:100170006A2500308A0051088207C528C928D000A6
:100180008A15FA238A111F26A628013049253830FE
:10019000BF286B304925013049253C30BF283B261C
:1001A0008316031318309200831203139D01143039
:1001B000B600F124043092000F309D04013090000D
:1001C0009601F93095000B30970083160313043025
:1001D0008C0083120313C0308B0087126423112517
:1001E000112511251125112511251125112511255F
:1001F000252394230038031DFF28EE231329013AF9
:10020000031D0729462300380319FD28ED285D2327
:100210000038031DED286125553049256825173024
:100220006A250825ED288716642311251125112537
:10023000112511251125112511251125252394237B
:100240000038031D2529EE233C29013A031D3029DE
:100250003823003803192329013A031DED281329F7
:1002600056230038031D1329612549304925682587
:1002700017306A25082513295D30EB000C30071F65
:100280000830EC0013236130EB00132302307002BE
:10029000031D4D290030EC00532903307002031D6B
:1002A00059290430EC005D30EB0013236130EB0082
:1002B00013233C30071F3830EC005530EB001E2371
:1002C0005930EB001E2302306F02031D6A290030F3
:1002D000EC00702903306F02031D76290430EC0016
:1002E0005530EB0013235930EB001323831603130F
:1002F00034304A020319C32983120313351E992986
:100300003512831603134A1A8C2983120313B51569
:10031000F4017414B516C329CA1A9229831203135F
:10032000B51188294A19C329831203134030B50631
:10033000C329B51EAB29B512831603134A19AB297D
:10034000D024612532306A25831603133430CA0065
:1003500083120313072B831603134A088312031314
:10036000C5004519B6290430B5067F23451ABA29B8
:100370000830B506C51AC329741EC1290130F4001E
:10038000C3290310F40D831603133430CA008312FB
:100390000313B51ECF29B51961242824D129282497
:1003A0007A246125B51DE029741CD729EC29F41C99
:1003B000DA293B2A741DDD29272AF41DD82AC82AE8
:1003C000741CE3295D2AF41CE629B42A741DE9296A
:1003D000922AF41DD82AC82A52304925703049255E
:1003E0006825AD308A15702465304724B7218A11FD
:1003F000B825013049253325E81F152AE8131430A4
:10040000351D10308A15FA2369304A2459214624B3
:10041000AD307024B7218A114C3049257030492500
:100420006825B82548304925ED2A1430351D10308F
:100430008A15FA2369304A24B7218A1143304925A5
:10044000703049256825B82546304925ED2A4730C2
:1004500049257030492568256530E8225330492503
:100460003325423049257030492568256930E82216
:1004700053304925ED2A52304925703049256825E9
:10048000AD308A15702465304724B7218A11B8250C
:1004900001304925332558304925703049256825D4
:1004A000AD308A15702469304724B7218A11803015
:1004B000A706B82501304925ED2A52304925733069
:1004C000492568256530E822013049253325E81F94
:1004D000802AE8131430351D10308A15FA2369304C
:1004E0004A2459214624AD307024B7218A11433063
:1004F0004925733049256825B82546304925ED2A18
:100500001430351D10308A15FA2369304A24B7217A
:100510008A114C304925733049256825B825483063
:100520004925ED2A47304925733049256825AD30E6
:100530008A15702465304724B7218A11B8255330B5
:100540004925332542304925733049256825AD308A
:100550008A15702469304724B7218A118030A70694
:10056000B82553304925ED2A5230492573304925A5
:1005700068256530E8220130492533255830492562
:100580007330492568256930E82201304925ED2A74
:100590005130492568258A1569304A246530472439
:1005A000B7217F30A7058A11B825B51D662AFB291A
:1005B0004430492568258A1565304A246930472426
:1005C000B7217F30A7058A11B825B51D662AFB29FA
:1005D0008A154A248A11B8250800351FF92ACD301A
:1005E00034254B30071F013049256F084725700817
:1005F00047258D3034253D30351D39306A25B51EEF
:10060000072BCB3034252630B51D2C306A258316B8
:100610000313CD0F0E2B83120313871383120313BF
:1006200035190825ED286C088A15FA238A156B08F8
:100630004A2459216B0842248A1108006C088A1543
:10064000F723002046248A11162B8A15E2238A11EB
:10065000A03084001430C9002830EA003514351861
:100660002F2B080083160313CD01831203130800F8
:1006700003307002031D432B071B0034322307177E
:100680000130F00002343223F00A01340230071F37
:1006900003306F02031D532B071F0034322307134F
:1006A0000130EF0002343223EF0A013401307002CE
:1006B000031900343223F003013401306F020319AF
:1006C00000343223EF0301347008871E6F08C50021
:1006D0006F30C50703300318013E8A0045088200C9
:1006E000732B772B7B2B0711752B871108000715B0
:1006F000792B8711080007157D2B871508005030CE
:10070000351D083083160313CC0083120313351DE7
:100710008E2B9601F93095000716080009309600D7
:10072000C330950007120800A03084000008D100F3
:10073000CF00840A0008D000CE00840A51080002CD
:10074000031CE22B031DAA2B840A50080002031C81
:10075000E52B840300084F02031CE82B031DB62B76
:10076000840A00084E02031CEB2BB72B840AC73007
:100770000402031D9D2B8A15EE235108A600500884
:10078000A5000020C5307524D8228A110038031D29
:1007900002348A15C93075244C238A110038031D90
:1007A00002348A154624EE234F08A6004E08A50001
:1007B00000204C22CD307524D8228A110038031D28
:1007C000013400340008D100840A0008D000B72B9F
:1007D0000008CF00840A0008CE00B72B8A15E72353
:1007E000EA0107308A0078306A0700278A155C24FE
:1007F0008624002059214D3047244E224D3042247A
:1008000007308A008C306A0700278A155C2486240A
:1008100000205921513047244E22513042248A1160
:10082000EA0A14306A02031DF12B4D30C6005D3018
:10083000871E5530C5008A154D248A115130C600D7
:100840006130871E5930C5008A154D248A11080071
:100850008A155D304A2446245921513042246130A2
:100860004A2446245921513047244E2251304224F3
:1008700055304A245D30472459214D3042245930A7
:100880004A246130472459214D3047244E225130AB
:100890004724B7216530422455304A24613047242B
:1008A00059214D3042245D304A2459304724592182
:1008B0004D3047244C2251304724B721693042241F
:1008C0008A115930C5006130C6000830C3004508A0
:1008D00084000008CC00460884000008CB004C08C7
:1008E0008000450884004B088000C503C603C30B85
:1008F000672C08008A1565304A248A112830351D76
:1009000018308A15FA234C225530422469304A2483
:100910008A112C30351D1C308A15FA234C2259308F
:10092000422465304A248A113030351D20308A1522
:10093000FA2359215D30422469304A248A11343027
:10094000351D24308A15FA23592146245D304A2466
:100950004C224624AD3070244C225D304224653058
:100960004A248A113430351D24308A15FA2359213E
:100970006130422469304A248A113030351D2030DC
:100980008A15FA235921462461304A244E228030A8
:10099000A706613042248A11B51961242824080071
:1009A0008312031365308A154A248A11351DDC2C05
:1009B0003030B51D2830DF2C2030B51D18308A1599
:1009C000172469304A248A11351DEA2C3430B51DAC
:1009D0002C30ED2C2430B51D1C308A1517248A11BB
:1009E000080007308A003603DA27B700CF309D05AC
:1009F000B70C03181D16B70C03189D1637083F399E
:100A00009B00B60B062D1430B6000800000008004D
:100A1000831203135930B8006230B9000230BA00B3
:100A2000232D831203131A30B8000630B9000030AA
:100A3000BA00232D831203133E30B8000030B900F2
:100A40000030BA00232DFF30B80703180301B9079F
:100A500003180301BA0703180301380439043A04E0
:100A6000031D232D0800C030C200420E0F3986003E
:100A70008616000000000000861242080F3986002A
:100A8000861600000000000086121A2508000F39A3
:100A90003038C200420E0F3910388600861600002A
:100AA00000000000861242080F39103886008616B2
:100AB000000000000000861286011A25080002309E
:100AC000622D01303425112D2E30492D3030492D25
:100AD0002030492DC300C30307308A004308002794
:100AE000FF39031908004925C30A6E2D4830342503
:100AF00007308A001030C3000030C40000274925A9
:100B0000C40A4408C30B7E2D08008400000E47254C
:100B1000000847253B300402031908008403862D92
:100B20002030C100BB01BC01BD01BE01BF01A40D4D
:100B3000A50DA60DA70DBB0DBC0DBD0DBE0DBF0DAA
:100B4000C10BA32D08000530C4003B308400A92D43
:100B5000840AAD25C40BA82D972D03300007C000D3
:100B6000C019800030300007C000C01B80000800A2
:100B7000A71FBD2DA7132D304925D101A130D000CD
:100B800050088A1575244C238A110038031DD02D76
:100B90000430D007D10A08305102031DC02DD10303
:100BA000510AD0000310D00DD00DA13050078A1586
:100BB0007524B721E8208A119025B5170430C800A4
:100BC0003F3005263F3005263E3005263E300526BF
:100BD0003D3005263D300526B5133C300526C808B6
:100BE0000319F92D64253C3002263B3002263B30A8
:100BF0000226B51E6825D030510700270038031D96
:100C0000492D0800C808031908008400800E000858
:100C1000B51F0E2E0F3903190800B513C8080319A4
:100C2000662DC8030008472508003515AC0A0319CE
:100C3000AD0A1F2E3515AC080319AD03AC032F30D8
:100C4000C6002730C5008A154D248A11B51304301B
:100C5000C800902533253C30052664253C30052608
:100C60003B3005263B3005260825080050088A152C
:100C700014248A1108008312031389309F001A2557
:100C80001F151F19412E81309F008A15EE238316F0
:100C900003131E0883120313A5001E08A6000020DC
:100CA0004030FA2359218A1111306A25B82556306F
:060CB0004925082508009B
:100E0000820700340E341134113411340A341B3487
:100E10000034003400341234123412341E341134CD
:100E2000103455346234613474343D340034413408
:100E30004434433420346F347634653472346C3443
:100E40006F346134643465346434003420346F3476
:100E5000703465346E340034733468346F347234F3
:100E6000743400345334613476346534643421345A
:100E700000343134303430340034203431346B3485
:100E80000034413444344A342034523473346834A6
:100E90003D3431343034303400347F340034003465
:100EA00000347E347334783471347E344F341B34E0
:100EB000BD347E341634793418347D341E343734DE
:100EC0007A3400340034003400347D349E343734B6
:100ED0007A347E349634793418347E34CF341B34EB
:100EE000BD347E34F334783471347F34803400344C
:100EF000003400340134023403340434053406343D
:100F00000734083409340A34093408340734063401
:100F10000534043403340234013405340634073410
:100F2000083409340A3409340834073406340534E3
:100F30000434033402340134003401340234033401
:100F400004349C346E346B34283492347434243436
:100F5000003488347A34003400347F340034003470
:100F600000347534033412346F346B340634373440
:100F7000BD346134093470345F3457340C34BC34BC
:100F8000CC344D3410341D347D3485342034003459
:100F900000348E341F34B03400348A346D348034DD
:100FA000003447344D346B3400346D3402346E34C5
:100FB000703466348207243418340E340734053410
:100FC00007340E3418342434323440344C3456341C
:0E0FD0005D345F345D3456344C34403432347A
:101000009630A800A901A71F0E28A509A609A709BF
:10101000A50A0319A60A0319A70AA917B3012708E5
:10102000031D23282608A7002508A600A501B3153F
:101030002708031D23282608A700A601B31133168D
:101040002708031934283308A802031D031C3F2A6C
:101050000310A71B3128A50DA60DA70DA80B292845
:101060003F2AA91FA7130034A701A601A501A401C7
:10107000A80100349E30A800A901A71F4B28A4098D
:10108000A509A609A709A40A0319A50A0319A60A0E
:101090000319A70AA917B3012708031D6B282608FF
:1010A000A7002508A6002408A500A401B315270859
:1010B000031D6B282608A7002508A600A501B3116B
:1010C00033162708031D6B282608A700A601B315B1
:1010D0002708031934283308A802031D031C3F2ADC
:1010E0000310A71B7A28A40DA50DA60DA70DA80B0C
:1010F00071283F2A2A1B251C3128A41F3128A50A44
:101100000319A60A0319A70A031D3128A70CA60C68
:10111000A50CA80A0319AC293128280803190034A2
:101120002708A900A7179630A802A81FDC28A8093D
:10113000A80A08302802031CB828A800A50D260814
:10114000A5002708A600A70108302802031CB8281C
:10115000A800A50D2608A500A60108302802031C3A
:10116000B828A800A50DA5012808031D0310C12853
:1011700028080319C1280310A70CA60CA50CA80B5E
:10118000BB282A1B251CCD28031CCD28A50A031922
:10119000A60A0319A70AA71BDC28A91F0034A70960
:1011A000A609A509A50A0319A60A0319A70A003466
:1011B000A701A601A50100342A14AA1FFF34A70124
:1011C000A91FFF30A700A600A500A90DA70CFF349A
:1011D000A4012808031900342708A900A7179E3086
:1011E000A802A81F4C29A809A80A08302802031C35
:1011F0002129A800A40D2508A4002608A500270879
:10120000A600A70108302802031C2129A800A40D6C
:101210002508A4002608A500A60108302802031C02
:101220002129A800A40D2508A400A5010830280242
:10123000031C2129A800A40DA4012808031D0310E4
:101240002B29280803192B290310A70CA60CA50C81
:10125000A40CA80B24292A1B241C3929031C392976
:10126000A40A0319A50A0319A60A0319A70AA71BAA
:10127000DC28A91F0034A709A609A509A409A40A06
:101280000319A50A0319A60A0319A70A0034A7011E
:10129000A601A501A40100342A14AA1FFF34A70146
:1012A000A91FFF30A700A600A500A400A90DA70C48
:1012B000FF342808031D2F080319342827082E0699
:1012C000A9002F08A8077E30031C6A29A80203186A
:1012D000AC296D29A802031C3F2A2708A400260870
:1012E000A3002508A200A417AE170310A701A601AA
:1012F000A5011830B300221C87292C08A5072D084A
:1013000003182D0FA6072E0803182E0FA707A70CEA
:10131000A60CA50CA40CA30CA20C0310B30B7B29E8
:10132000A71B9729A40DA50DA60DA70DA8032A1B81
:10133000251CA929A41FA929A50A0319A60A03196E
:10134000A70A031DA929A70CA60CA50CA80A031916
:10135000AC29A91FA7130034AA14AA1FFF34FF3019
:10136000A800A700A600A500A90DA70CFF342F0810
:1013700003194A2A28080319342827082E06A90029
:10138000A717AE17B3012708A4002608A300250855
:10139000A2002C08A2022D08031C2D0FA3022E0868
:1013A000031C2E0FA402A401A301A201031CDF2928
:1013B0000310A70CA60CA50CA40C0130B3002F0839
:1013C000A802031CE9297E303307A8070318AC29BB
:1013D000EE297E303307A807031C3F2A1830B200DD
:1013E000A20DA30DA40DA50DA60DA70DB30D2C08E0
:1013F000A5022D08031C2D0FA6022E08031C2E0F7C
:10140000A7022E0DB304331C072A2214122A2C081B
:10141000A5072D0803182D0FA6072E0803182E0A5E
:10142000A7072210B20BF0292A1B221C362A031010
:10143000A50DA60DA70DB30D2C08A5022D08031CA4
:101440002D0FA6022E08031C2E0FA7022E0D33040B
:101450000139A2070318A30A0319A40A031D362A97
:10146000A40CA30CA20CA80A0319AC29A91FA4134D
:101470002408A7002308A6002208A50000342A1586
:10148000AA1FFF340130A800A701A601A501A90DDC
:10149000A70CFF34AA15FF348030AE0627082E06AD
:1014A000B300A401AB0128082F02031C6F2A2F08E8
:1014B000A2002808AF002208A8002E08A2002708D2
:1014C000AE002208A7002D08A2002608AD002208C1
:1014D000A6002C08A2002508AC002208A5002F08B1
:1014E000031900342708A900A717AE172F082802F0
:1014F000AF000319A22A08302F02031C982AAF005C
:101500002C08AB002D08AC002E08AD00AE01083051
:101510002F02031C982AAF002C08AB002D08AC004A
:10152000AD0108302F02031C982A2908A7000034B7
:101530002F080319A22A0310AE0CAD0CAC0CAB0C97
:10154000AF0B9B2AB31FAF2AAB09AC09AD09AE099B
:10155000AB0A0319AC0A0319AD0A0319AE0A2B082A
:10156000A4072C0803182C0FA5072D0803182D0F0E
:10157000A6072E0803182E0FA707B31BC82A031CA3
:101580007A28A70CA60CA50CA40CA80F7A28AC29C5
:1015900003184B28A409A509A609A709A40A031939
:1015A000A50A0319A60A0319A70A8030A9060E285E
:1015B00027082E06B300B31B112BA71BF82A2808F7
:1015C0002F02031C0034031D013427082E02031CC4
:1015D0000034031D013426082D02031C0034031DB2
:1015E000013425082C02031C0034031D013400348F
:1015F0002F082802031C0034031D01342E08270283
:10160000031C0034031D01342D082602031C003482
:10161000031D01342C082502031C0034031D013472
:101620000034AE1F0134003427082E06B300B31B6C
:10163000492BA71B322B28082F02031C0034031D43
:10164000013427082E02031C0034031D0134260830
:101650002D02031C0034031D013425082C02031C39
:10166000003401342F082802031C0034031D013408
:101670002E082702031C0034031D01342D08260206
:10168000031C0034031D01342C082502031C003404
:101690000134AE1F013400342E082706B300B31BFB
:1016A000852BAE1B6C2B2F082802031C0034031D56
:1016B00001342E082702031C0034031D01342D08B9
:1016C0002602031C0034031D01342C082502031CD0
:1016D0000034031D0134003428082F02031C003499
:1016E000031D013427082E02031C0034031D01349E
:1016F00026082D02031C0034031D013425082C028A
:10170000031C0034031D01340034A71F01340034CE
:101710002E082706B300B31BBD2BAE1BA62B2F082C
:101720002802031C0034031D01342E082702031C69
:101730000034031D01342D082602031C0034031D50
:1017400001342C082502031C0034013428082F0220
:10175000031C0034031D013427082E02031C00342F
:10176000031D013426082D02031C0034031D01341F
:1017700025082C02031C00340134A71F0134003457
:101780002F082802031D00342E082702031D0034F1
:101790002D082602031D00342C082502031D0034E9
:1017A00001342F082802031D01342E082702031DCF
:1017B00001342D082602031D01342C082502031DC7
:1017C00001340034C73084002830C300F22B51307C
:1017D00084000830C300F22B2F30EF2B2830840018
:1017E0000430C30080018403C30BF22B0800ED001A
:1017F0002830FC2BED002F3084000430C300082477
:10180000831203138000ED0A8403C30BFF2B08002F
:101810006D08831203178D00831603178C130C14A5
:10182000831203170C080800ED002F30192CED006F
:10183000283084000430C3000008EE002624831200
:101840000313ED0A8403C30B1C2C08008316031733
:101850008C18282C831203136D08831203178D0034
:10186000831203136E08831203178C008316031769
:101870008C130C1555308D00AA308D008C1400008F
:101880000C110800C5002830C6004D2C2830C600B9
:101890002F304C2CC6002830C5000430C300460849
:1018A00084000008C7004508840047088000C5037D
:1018B000C603C30B4F2C0800EB000310EB0DEB0D20
:1018C0002F3084000430C30007308A004C306B078F
:1018D00000278A158000EB0A8403C30B642C0800E0
:1018E000EB00EB0328308400792CEB00EB032F3066
:1018F00084000430C30007308A006B0800278A1573
:101900008000EB0A8403C30B7B2C0800EE236A08DB
:10191000EB000310EB0DA0306B0784000008A6005D
:08192000840A0008A50008007C
:02400E00323F3F
:104200007B004C00CC00CD0078002300D7000A00D2
:10421000810024001A00420078002300D7000A0021
:1042200088001D00140062008B00440059007C00CF
:10423000000000000000000000000000000000007E
:10424000000000000000000000000000000000006E
:10425000000000000000000000000000000000005E
:10426000000000000000000000000000000000004E
:10427000003400340334E834003400340334E834C8
:08428000793416342834CC34E3
:00000001FF
